:020000040000FA
:0400000022EF0BF0F0
:06002A00D9CFE5FFE1CF94
:10003000D9FF00C0E5FF01C0E5FF02C0E5FF03C036
:10004000E5FF04C0E5FF05C0E5FF06C0E5FF07C00A
:10005000E5FF08C0E5FF09C0E5FF0AC0E5FF020EA5
:10006000DBCF00F0030EDBCF01F0040EDBCF02F09C
:10007000050EDBCF03F0060EDBCF04F0070EDBCF5F
:1000800005F000C006F001C007F002C008F0035000
:1000900003E003500508036E270EE56E100EE56EB3
:1000A0000550E56E0450E56E46EC05F0096EF3CFA1
:1000B0000AF0040EE126300E092609C0E5FF06C04D
:1000C000E9FF07C0F3FF085038EC0BF0062AD8B060
:1000D000072AD8B0082A030603500EE12E0EE56E5B
:1000E00006C0E9FF07C0F3FF085038EC0BF0062A02
:1000F000D8B0072AD8B0082A270EE56E100EE56E94
:100100000550E56E0450E56EEAEC04F0046EF3CFA2
:1001100005F0040EE126030EE56EE80EE56E0550CF
:10012000E56E0450E56E46EC05F0096EF3CF0AF07B
:10013000040EE126300E092609C0E5FF06C0E9FFDE
:1001400007C0F3FF085038EC0BF0062AD8B0072A96
:10015000D8B0082A030603500EE12E0EE56E06C045
:10016000E9FF07C0F3FF085038EC0BF0062AD8B0BF
:10017000072AD8B0082A030EE56EE80EE56E055092
:10018000E56E0450E56EEAEC04F0046EF3CF05F082
:10019000040EE126000EE56E640EE56E0550E56E78
:1001A0000450E56E46EC05F0096EF3CF0AF0040E3C
:1001B000E126300E092609C0E5FF06C0E9FF07C0A9
:1001C000F3FF085038EC0BF0062AD8B0072AD8B055
:1001D000082A030603500EE12E0EE56E06C0E9FF65
:1001E00007C0F3FF085038EC0BF0062AD8B0072AF6
:1001F000D8B0082A000EE56E640EE56E0550E56E77
:100200000450E56EEAEC04F0046EF3CF05F0040E42
:10021000E126000EE56E0A0EE56E0550E56E04500F
:10022000E56E46EC05F0096EF3CF0AF0040EE12608
:10023000300E092609C0E5FF06C0E9FF07C0F3FF3D
:10024000085038EC0BF0062AD8B0072AD8B0082A94
:10025000030603500EE12E0EE56E06C0E9FF07C04F
:10026000F3FF085038EC0BF0062AD8B0072AD8B0B4
:10027000082A000EE56E0A0EE56E0550E56E045084
:10028000E56EEAEC04F0046EF3CF05F0040EE1260F
:10029000300E042604C0E5FF06C0E9FF07C0F3FFE7
:1002A000085038EC0BF0062AD8B0072AD8B0082A34
:1002B000032E09D02E0EE56E06C0E9FF07C0F3FF3E
:1002C000085038EC0BF00050040F036E000E0120B4
:1002D000046E000E0220056E0250800FF36E055072
:1002E000800FF35C05E10450015C02E10350005C07
:1002F0001AE200C0E9FF01C0F3FF02509DEC0AF0D2
:10030000066E0650300A0FE1200EE56E00C0E9FFD0
:1003100001C0F3FF025038EC0BF0002AD8B0012ADC
:10032000D8B0022AD9D7E4CF0AF0E4CF09F0E4CF5D
:1003300008F0E4CF07F0E4CF06F0E4CF05F0E4CF17
:1003400004F0E4CF03F0E4CF02F0E4CF01F0E4CF17
:1003500000F0E4CFD9FF1200D9CFE5FFE1CFD9FFFC
:1003600000C0E5FF01C0E5FF02C0E5FF03C0E5FFF7
:1003700004C0E5FF05C0E5FF06C0E5FF07C0E5FFD7
:10038000020EDBCF00F0030EDBCF01F0040EDBCF5B
:1003900002F0050EDBCF03F0640EE56E03C0E5FF4F
:1003A000AFEC08F0046EE450E450300E042604C0B4
:1003B000E5FF00C0E9FF01C0F3FF025038EC0BF08D
:1003C0000050010F046E000E0120056E000E022089
:1003D000066E640EE56E03C0E5FF75EC08F0036E73
:1003E000E450E4500A0EE56E03C0E5FFAFEC08F000
:1003F000076EE450E450300E072607C0E5FF04C046
:10040000E9FF05C0F3FF065038EC0BF0042AD8B022
:10041000052AD8B0062A0A0EE56E03C0E5FF75EC82
:1004200008F0036EE450E450300E032603C0E5FFED
:1004300004C0E9FF05C0F3FF065038EC0BF0005094
:10044000020F036E000E0120046E000E0220056EE6
:100450000250800FF36E0550800FF35C05E10450ED
:10046000015C02E10350005C1AE200C0E9FF01C038
:10047000F3FF02509DEC0AF0066E0650300A0FE1C1
:10048000200EE56E00C0E9FF01C0F3FF025038EC1A
:100490000BF0002AD8B0012AD8B0022AD9D7E4CF6D
:1004A00007F0E4CF06F0E4CF05F0E4CF04F0E4CFAA
:1004B00003F0E4CF02F0E4CF01F0E4CF00F0E4CFAA
:1004C000D9FF1200D9CFE5FFE1CFD9FF00C0E5FF8A
:1004D00001C0E5FF02C0E5FF03C0E5FF04C0E5FF82
:1004E00005C0E5FF06C0E5FF07C0E5FF08C0E5FF62
:1004F000020EDBCF00F0030EDBCF01F0040EDBCFEA
:1005000002F0050EDBCF03F0060EDBCF04F0070E82
:10051000DBCF05F0080EDBCF06F0090EDBCF07F0CE
:1005200081EC09F003A003D0020EC86E02D0090EC0
:10053000C86E16EC0BF00050E56EF2EC0AF0E12A02
:1005400003A208D00250036E086A0350E56EF2EC75
:100550000AF0E12A0150E56EF2EC0AF0E12A0AEC19
:100560000BF000800050E56EF2EC0AF0E12A04C0C6
:1005700000F005C001F006C002F007C003F0020E53
:10058000035C16E3010EE56EFCEC09F0046EE12A53
:1005900004C0E5FF00C0E9FF01C0F3FF025038ECE2
:1005A0000BF0002AD8B0012AD8B0022A0306E7D7F8
:1005B00003500FE0000EE56EFCEC09F0036EE12A3B
:1005C00003C0E5FF00C0E9FF01C0F3FF025038ECB3
:1005D0000BF0FEEC0AF0E86AE4CF08F0E4CF07F095
:1005E000E4CF06F0E4CF05F0E4CF04F0E4CF03F06D
:1005F000E4CF02F0E4CF01F0E4CF00F0E4CFD9FF84
:100600001200D9CFE5FFE1CFD9FF00C0E5FF01C05F
:10061000E5FF02C0E5FF03C0E5FF04C0E5FF05C03C
:10062000E5FF06C0E5FF07C0E5FF08C0E5FF09C01C
:10063000E5FF0AC0E5FF0BC0E5FF0CC0E5FF0DC0FC
:10064000E5FF020EDBCF00F0030EDBCF01F0040E5E
:10065000DBCF02F0050EDBCF03F0060EDBCF04F09C
:10066000070EDBCF05F0080EDBCF06F0090EDBCF5F
:1006700007F0086A096A0A6A0B6A200E0C6E0344C6
:10068000010B0D6E010E0D160050002601360236CC
:1006900003360850082609360A360B360D50D8A402
:1006A000088007500B5C08E106500A5C05E1055024
:1006B000095C02E10450085C09E30450085E05503F
:1006C000095A06500A5A07500B5A00800C2ED7D7E9
:1006D00003C0E9FF02C0F4FF01C0F3FF0050E4CF04
:1006E0000DF0E4CF0CF0E4CF0BF0E4CF0AF0E4CF50
:1006F00009F0E4CF08F0E4CF07F0E4CF06F0E4CF50
:1007000005F0E4CF04F0E4CF03F0E4CF02F0E4CF4F
:1007100001F0E4CF00F0E4CFD9FF1200D9CFE5FF1C
:10072000E1CFD9FF00C0E5FF01C0E5FF02C0E5FF52
:1007300003C0E5FF04C0E5FF05C0E5FF06C0E5FF17
:1007400007C0E5FF020EDBCF00F0030EDBCF01F0A8
:10075000040EDBCF02F0050EDBCF03F0060EDBCF7D
:1007600004F0070EDBCF05F0080EDBCF06F0090E14
:10077000DBCF07F081EC09F003A003D0020EC86EB6
:1007800002D0090EC86E16EC0BF00050E56EF2ECCC
:100790000AF0E12A03A208D00250006E036A00505A
:1007A000E56EF2EC0AF0E12A0150E56EF2EC0AF097
:1007B000E12A04C000F005C001F006C002F007C045
:1007C00003F003C004F00306045013E000C0E9FF87
:1007D00001C0F3FF02509DEC0AF0046E002AD8B06D
:1007E000012AD8B0022A0450E56EF2EC0AF0E12AA0
:1007F000E8D7FEEC0AF0E86AE4CF07F0E4CF06F0B1
:10080000E4CF05F0E4CF04F0E4CF03F0E4CF02F04E
:10081000E4CF01F0E4CF00F0E4CFD9FF1200D9CF4C
:10082000E5FFE1CFD9FF00C0E5FF01C0E5FF02C051
:10083000E5FF03C0E5FF04C0E5FF020EDBCF00F0DB
:10084000030EDBCF01F0040EDBCF02F0050EDBCF91
:1008500003F0060EDBCF04F081EC09F0090EC86E40
:1008600016EC0BF0C60EE56EF2EC0AF0E12A000E73
:10087000E56EF2EC0AF0E12AFE0EE56EF2EC0AF00B
:10088000E12A0150400DF3CF01F0800E0126015006
:1008900000260050E56EF2EC0AF0E12A02C000F0FA
:1008A00003C001F004C002F000C0E9FF01C0F3FF83
:1008B00002509DEC0AF0036E03500BE0002AD8B002
:1008C000012AD8B0022A0350E56EF2EC0AF0E12AC0
:1008D000EBD7FF0EE56EF2EC0AF0E12AFEEC0AF02F
:1008E000000EE56E0A0EE56E4FEC09F0020EE126F1
:1008F000E4CF04F0E4CF03F0E4CF02F0E4CF01F062
:10090000E4CF00F0E4CFD9FF1200D9CFE5FFE1CF6B
:10091000D9FF00C0E5FF01C0E5FF02C0E5FF03C04D
:10092000E5FF04C0E5FF05C0E5FF06C0E5FF07C021
:10093000E5FF08C0E5FF09C0E5FF0AC0E5FF0BC001
:10094000E5FF020EDBCF00F00050E56E01EC08F091
:10095000016EF3CF02F0E12A036A046A002A002A3A
:100960000050E56E01EC08F0006EF3CF05F0E12ACF
:10097000066A076A05500B6E00500A6E086A096A1B
:1009800008500112095002120A5003120B500412AF
:1009900004C0E9FF03C0F4FF02C0F3FF0150E4CF3D
:1009A0000BF0E4CF0AF0E4CF09F0E4CF08F0E4CF95
:1009B00007F0E4CF06F0E4CF05F0E4CF04F0E4CF95
:1009C00003F0E4CF02F0E4CF01F0E4CF00F0E4CF95
:1009D000D9FF1200D9CFE5FFE1CFD9FF00C0E5FF75
:1009E00001C0E5FF02C0E5FF03C0E5FF04C0E5FF6D
:1009F00005C0E5FF06C0E5FF020EDBCF00F0030EE9
:100A0000DBCF01F0040EDBCF02F0050EDBCF03F0ED
:100A1000046A056A0344010B066E06B011D0025049
:100A2000022603360350015C02E10250005C04E23E
:100A3000D8900332023204D0052A05C004F0EAD768
:100A40000350015C02E10250005C04E30250005ECE
:100A50000350015AD8900332023204C005F0040654
:100A60000550EEE101C0F3FF0050E4CF06F0E4CF03
:100A700005F0E4CF04F0E4CF03F0E4CF02F0E4CFDC
:100A800001F0E4CF00F0E4CFD9FF1200D9CFE5FFA9
:100A9000E1CFD9FF00C0E5FF01C0E5FF02C0E5FFDF
:100AA00003C0E5FF04C0E5FF05C0E5FF06C0E5FFA4
:100AB00007C0E5FF020EDBCF00F0030EDBCF01F035
:100AC000040EDBCF02F0050EDBCF03F0046A056AEB
:100AD000100E066E0144010B076E010E0716005042
:100AE000002601360450042605360750D8A4048099
:100AF0000350055C02E10250045C05E30250045E11
:100B00000350055A0080062EE5D701C0F3FF0050C0
:100B1000E4CF07F0E4CF06F0E4CF05F0E4CF04F033
:100B2000E4CF03F0E4CF02F0E4CF01F0E4CF00F033
:100B3000E4CFD9FF1200D9CFE5FFE1CFD9FF00C044
:100B4000E5FF01C0E5FF02C0E5FF020EDBCF00F0CC
:100B500000380F0B016E300E01263A0E015C02E3E5
:100B6000070E012601500001876F0F0E0014016E61
:100B7000300E01263A0E015C02E3070E01260150F9
:100B80000001886F00018969000E016E870E006EFA
:100B9000800E026E030EE56E0250E56E0150E56EAA
:100BA0000050E56E000EE56E000EE56E000EE56E7F
:100BB000C60EE56E8EEC03F0080EE126000EE56E23
:100BC0000A0EE56E4FEC09F0020EE126E4CF02F0CA
:100BD000E4CF01F0E4CF00F0E4CFD9FF1200D9CF89
:100BE000E5FFE1CFD9FF00C0E5FF01C0E5FF02C08E
:100BF000E5FF03C0E5FF04C0E5FF05C0E5FF06C053
:100C0000E5FF020EDBCF00F0030EDBCF01F0040E98
:100C1000DBCF02F0050EDBCF03F0060EDBCF04F0D6
:100C20000150056E0250066E0650E56E0550E56EE9
:100C30000050E56EC6EC07F0030EE126002A002AFC
:100C40000350016E0450026E036A046A0250E56E9E
:100C50000150E56E0050E56EC6EC07F0030EE1268C
:100C6000E4CF06F0E4CF05F0E4CF04F0E4CF03F0E6
:100C7000E4CF02F0E4CF01F0E4CF00F0E4CFD9FFFD
:100C80001200840EF66E160EF76E000EF86E090056
:100C9000F550056E0900F550066E055002E106504C
:100CA0003BE00900F550006E0900F550016E0900A7
:100CB000F550026E09000900F550E96E0900F55083
:100CC000EA6E090009000900F550036E0900F550AD
:100CD000046E09000900F6CF07F0F7CF08F0F8CF4F
:100CE00009F000C0F6FF01C0F7FF02C0F8FF035093
:100CF00002E1045007E00900F550EE6E0306F8E249
:100D00000406F9D707C0F6FF08C0F7FF09C0F8FFCF
:100D10000506C4E20606C5D71200D9CFE5FFE1CF2C
:100D2000D9FF00C0E5FF01C0E5FF02C0E5FF03C039
:100D3000E5FF04C0E5FF05C0E5FF020EDBCF00F0D4
:100D4000030EDBCF01F0040EDBCF02F0050EDBCF8C
:100D500003F0046A0350045C14E200C0E9FF01C020
:100D6000F3FF02509DEC0AF0056E002AD8B0012A6C
:100D7000D8B0022A0550E56E8BEC0AF0E12A042A6D
:100D8000E9D7E4CF05F0E4CF04F0E4CF03F0E4CFFB
:100D900002F0E4CF01F0E4CF00F0E4CFD9FF12007D
:100DA000D9CFE5FFE1CFD9FF00C0E5FF01C0E5FFE6
:100DB00002C0E5FF03C0E5FFE6EC08F0006EF3CFEC
:100DC00001F0F4CF02F0E9CF03F0000EE56E0F0E54
:100DD000E56E420EE56E400EE56E0350E56E025084
:100DE000E56E0150E56E0050E56E01EC03F0006E1B
:100DF000F3CF01F0F4CF02F0E9CF03F0080EE126C3
:100E000001C0F3FF0050E4CF03F0E4CF02F0E4CFE1
:100E100001F0E4CF00F0E4CFD9FF1200D9CFE5FF15
:100E2000E1CFD9FF00C0E5FF01C0E5FF02C0E5FF4B
:100E300003C0E5FFE6EC08F0006EF3CF01F0F4CF5D
:100E400002F0E9CF03F0000EE56E000EE56E030E32
:100E5000E56EE80EE56E0350E56E0250E56E01505A
:100E6000E56E0050E56E01EC03F0006EF3CF01F08B
:100E7000F4CF02F0E9CF03F0080EE12601C0F3FF42
:100E80000050E4CF03F0E4CF02F0E4CF01F0E4CF70
:100E900000F0E4CFD9FF1200D9CFE5FFE1CFD9FFB1
:100EA00000C0E5FF01C0E5FF02C0E5FF020EDBCF99
:100EB00000F0005000018A6F00018B69000E016E86
:100EC0008A0E006E800E026E020EE56E0250E56E16
:100ED0000150E56E0050E56E000EE56E000EE56E09
:100EE000000EE56EC60EE56E8EEC03F0080EE126F0
:100EF000000EE56E0A0EE56E4FEC09F0020EE126DB
:100F0000E4CF02F0E4CF01F0E4CF00F0E4CFD9FF6A
:100F10001200D9CFE5FFE1CFD9FF00C0E5FF01C046
:100F2000E5FF02C0E5FFFE0E0001846F010E000127
:100F3000856F00018669000E016E840E006E800EC2
:100F4000026E030EE56E0250E56E0150E56E005034
:100F5000E56E000EE56E000EE56E000EE56EC60E47
:100F6000E56E8EEC03F0080EE126000EE56E0A0E2B
:100F7000E56E4FEC09F0020EE126E4CF02F0E4CF7B
:100F800001F0E4CF00F0E4CFD9FF1200D9CFE5FFA4
:100F9000E1CFD9FF00C0E5FF01C0E5FF02C0E5FFDA
:100FA000020EDBCF00F0030EDBCF01F0040EDBCF2F
:100FB00002F0A69EA69CA684F29E00C0A9FF015046
:100FC000A86E550EA76EAA0EA76EA682A6B2FED771
:100FD0000028A96E0250016E026A0150A86E550EDB
:100FE000A76EAA0EA76EA682A6B2FED7A694F28E10
:100FF000E4CF02F0E4CF01F0E4CF00F0E4CFD9FF7A
:101000001200D9CFE5FFE1CFD9FF00C0E5FF01C055
:10101000E5FF02C0E5FF03C0E5FF04C0E5FF05C032
:10102000E5FF020EDBCF00F0A69CA69E00C0A9FF44
:10103000A680A8CF01F0026A0028A96EA680A8CFDA
:1010400000F0036A0050056E046A04500112055056
:10105000021202C0F3FF0150E4CF05F0E4CF04F028
:10106000E4CF03F0E4CF02F0E4CF01F0E4CF00F0EE
:10107000E4CFD9FF1200D9CFE5FFE1CFD9FF00C0FF
:10108000E5FF01C0E5FF02C0E5FF03C0E5FF020E7A
:10109000DBCF00F0030EDBCF01F0040EDBCF02F05C
:1010A00000C0E9FF01C0F3FF02509DEC0AF0036E9F
:1010B000035010E0ACA2FED700C0E9FF01C0F3FF6F
:1010C00002509DEC0AF0AD6E002AD8B0012AD8B0CB
:1010D000022AE6D7E4CF03F0E4CF02F0E4CF01F038
:1010E000E4CF00F0E4CFD9FF1200D9CFE5FFE1CF84
:1010F000D9FF00C0E5FF01C0E5FF02C0E5FF03C066
:10110000E5FF020EDBCF00F0030EDBCF01F0026A39
:10111000036A01BE0CD0D89001360150005C03E296
:10112000D890013204D0032A03C002F0F2D7015054
:10113000005C02E30150005ED890013202C003F06F
:1011400002060350F4E10050E4CF03F0E4CF02F0D4
:10115000E4CF01F0E4CF00F0E4CFD9FF1200D9CF03
:10116000E5FFE1CFD9FF00C0E5FF01C0E5FF02C008
:10117000E5FF03C0E5FF04C0E5FF020EDBCF00F092
:10118000030EDBCF01F0026A080E036E800E00141E
:10119000046ED8900036D89002360450D8A402804D
:1011A0000150025C03E30150025E0080032EEED783
:1011B0000050E4CF04F0E4CF03F0E4CF02F0E4CF3A
:1011C00001F0E4CF00F0E4CFD9FF120000C0E5FF4A
:1011D00001C0E5FF02C0E5FF03C0E5FF04C0E5FF75
:1011E00005C0E5FFB2CF00F0B3CF01F08CC002F034
:1011F0008DC003F0B2CF04F0B3CF05F00150055C11
:1012000002E10050045C04E28CC002F08DC003F0E7
:1012100003C0E9FF02C0F4FF05C0F3FF0450E4CFB0
:1012200005F0E4CF04F0E4CF03F0E4CF02F0E4CF24
:1012300001F0E4CF00F01200D9CFE5FFE1CFD9FFF4
:1012400000C0E5FF01C0E5FF02C0E5FF03C0E5FF08
:10125000020EDBCF00F00044E844FC0B016E030EED
:101260000110C26EC2B2FED7C4CF00F0016A0050B6
:10127000036E026AC3CF00F0016A005002260150DB
:10128000032203C0F3FF0250E4CF03F0E4CF02F0E7
:10129000E4CF01F0E4CF00F0E4CFD9FF1200D9CFC2
:1012A000E5FFE1CFD9FF00C0E5FF01C0E5FF02C0C7
:1012B000E5FF03C0E5FF020EDBCF00F0030EDBCF3E
:1012C00001F000C002F001C003F0FF0E0026D8A01C
:1012D00001060250031006E0FA0E026E0000022E14
:1012E000FDD7EFD7E4CF03F0E4CF02F0E4CF01F075
:1012F000E4CF00F0E4CFD9FF120054657374696E37
:101300006700D9CFE5FFE1CFD9FF00C0E5FF01C0FD
:10131000E5FF02C0E5FFFF0E006E1F0EC514016E53
:10132000026AC7B4022A02500112015003E000060B
:101330000050F3E100C001F0005002E137EC0AF088
:101340000150D880E866D890016A01360150E4CF98
:1013500002F0E4CF01F0E4CF00F0E4CFD9FF1200B7
:10136000110E0001806F220E0001816F330E00010B
:10137000826F440E0001836F620ED36E0F0E936E68
:10138000816A818E62EC0AF089EC07F0000EE56E4E
:10139000120EE56EFA0EE56E010EE56E020EE56EBA
:1013A0000FEC04F0050EE126FFD71200D9CFE5FFC0
:1013B000E1CFD9FF00C0E5FF01C0E5FF020EDBCFA2
:1013C00000F0030EDBCF01F0A69EA69CA684F29E41
:1013D00001C0A8FF00C0A9FF550EA76EAA0EA76EF8
:1013E000A682A6B2FED7A694F28EE4CF01F0E4CF97
:1013F00000F0E4CFD9FF1200D9CFE5FFE1CFD9FF4C
:1014000000C0E5FF01C0E5FF020EDBCF00F081EC7C
:1014100009F0C58681EC09F0C9CF01F081EC09F033
:10142000005002E0C59A01D0C58AC5880150E4CFBA
:1014300001F0E4CF00F0E4CFD9FF1200D9CFE5FFEF
:10144000E1CFD9FF00C0E5FF01C0E5FF1F0EC514C5
:10145000006E016AC7B4012A015000120050F6E183
:10146000E4CF01F0E4CF00F0E4CFD9FF1200D9CFF0
:10147000E5FFE1CFD9FF818AC69A9496828682B829
:1014800003D082968286FBD794988298828894862D
:101490009488C68AE4CFD9FF1200D9CFE5FFE1CF07
:1014A000D9FF200EAC6E900EAB6E0C0EAF6E000E20
:1014B000E56E010EE56E4FEC09F0020EE126E4CF79
:1014C000D9FF1200D9CFE5FFE1CFD9FF3F0EC716F4
:1014D000280EC66EC56A090EC86E948694889E96BC
:1014E000A19637EC0AF0819AE4CFD9FF1200D9CF48
:1014F000E5FFE1CFD9FF00C0E5FF020EDBCF00F032
:10150000A69CA69E00C0A9FFA680A850E4CF00F02C
:10151000E4CFD9FF1200D9CFE5FFE1CFD9FF00C05A
:10152000E5FF020EDBCF00F0ACA2FED700C0ADFF9E
:10153000E4CF00F0E4CFD9FF1200E8AE04D0F3CF3F
:10154000EAFFEE501200E8BC08D0E9CFF6FFF3CF77
:10155000F7FFF86E0900F55012001200D9CFE5FF31
:10156000E1CFD9FF810EB16EB36AB26A00018C6B14
:1015700000018D6BE4CFD9FF1200D9CFE5FFE1CF99
:10158000D9FF00C0E5FF006A9EBA002A0050E4CFF0
:1015900000F0E4CFD9FF1200D9CFE5FFE1CFD9FFAA
:1015A000010EC26E050EC16E940EC06EE4CFD9FF5F
:1015B0001200D9CFE5FFE1CFD9FFB36AB26A0001CB
:1015C0008C6B00018D6BE4CFD9FF1200D9CFE5FF02
:1015D000E1CFD9FF00018C2B02E300018D2BE4CF7A
:1015E000D9FF1200D9CFE5FFE1CFD9FF020EDBCF43
:1015F000C9FF81EC09F0E4CFD9FF1200D9CFE5FF94
:10160000E1CFD9FF81EC09F0C584C5B4FED7E4CFA2
:10161000D9FF1200D9CFE5FFE1CFD9FF81EC09F066
:10162000C582C5B2FED7E4CFD9FF1200D9CFE5FFFE
:10163000E1CFD9FF81EC09F0C580C5B0FED7E4CF7A
:10164000D9FF120012EEFFF022EEFFF0F86AA68E2C
:10165000A69C41EC06F0B0EC09F0FFD7D9CFE5FF2E
:10166000E1CFD9FF9EAAFED7AE50E4CFD9FF12003A
:10167000E8AE05D0F3CFEAFFE4CFEEFF1200E8AC0E
:10168000120012000100921600008E0000000100FE
:041690000000000056
:00000001FF
